:100000001BC100001DC70000F0C60000C3C60000F1
:1000100096C6000069C600003CC600003DC1000055
:100020003BC1000039C1000037C1000035C10000EC
:1000300033C1000031C100002FC100002DC10000FC
:100040002BC1000029C1000027C1000025C100000C
:1000500023C1000021C100001FC10000D0C5000065
:100060001BC1000096C500006BC5000015C1000053
:1000700013C1000011C100000FC100000DC100003C
:100080000BC1000009C1000007C1000005C100004C
:1000900003C1000001C10000FFC00000FDC000005E
:1000A000FBC00000F9C00000F7C00000F5C0000070
:1000B000F3C00000F1C00000EFC00000EDC0000080
:1000C000EBC00000E9C00000E7C00000E5C0000090
:1000D000E3C00000E1C00000DFC00000DDC00000A0
:1000E000DBC00000000020002300260029002C00B7
:1000F0002F00320000010000030106010901000089
:100100002100240027002A002D00300033000101C7
:100110000000040107010A01000022002500280058
:100120002B002E00310034000201000005010801FF
:100130000B0105050505070508080808020202026B
:100140000A0A080804040404010101010101010173
:100150000303030303030303040707070C0C0C0C3E
:100160000C0C0C0C02020202060606060606060627
:100170000B0B0B0B0B0B0B0B0102102020080810B4
:100180002040102040800201020108040201010207
:1001900004081020408080402010080402018004E0
:1001A000020180402010080402010804020101023B
:1001B0000408102040800102040810204080000044
:1001C0000A0B02090C0D0E080703040100000000D1
:1001D000000000000000000000000000000000001F
:1001E00000000000000000000000121110000000DC
:1001F00000000000000000000000000000000000FF
:10020000000000003D300A003D310A000A003D3088
:100210000A003D310A000A000A000A0023002300F8
:100220002300232323235265616C53696D47656165
:1002300072230000E707600D11241FBECFEFD1E24B
:10024000DEBFCDBF00E00CBF26E0AEE6B4E001C0EB
:100250001D92A737B207E1F714E0A0E0B2E0E2E0B8
:10026000F0E200E00BBF02C007900D92AE36B1077E
:10027000D9F711E0CBE1D1E000E006C021970109F8
:10028000802FFE010E94CB0DCA31D10780E0080704
:10029000A9F76BD70C94F00FB3CEAF92BF92CF9269
:1002A000DF92EF92FF920F931F93CF93DF936C0136
:1002B0007B018B01040F151FEB015E01AE18BF0817
:1002C000C017D10759F06991D601ED91FC910190C9
:1002D000F081E02DC6011995892B79F7C501DF91D1
:1002E000CF911F910F91FF90EF90DF90CF90BF9033
:1002F000AF900895FC01538D448D252F30E0842F5D
:1003000090E0821B930B541710F0CF96089501973D
:100310000895FC01918D828D981761F0A28DAE0F2A
:10032000BF2FB11D5D968C91928D9F5F9F73928FB1
:1003300090E008958FEF9FEF0895FC01918D828DDD
:10034000981731F0828DE80FF11D858D90E00895AA
:100350008FEF9FEF0895FC01918D228D892F90E002
:10036000805C9F4F821B91098F73992708958BE9B9
:1003700094E0F1DF21E0892B09F420E0822F089539
:10038000FC01A48DA80FB92FB11DA35ABF4F2C910A
:10039000848D90E001968F739927848FA689B78901
:1003A0002C93A089B1898C91837080648C93938DF8
:1003B000848D981306C00288F389E02D80818F7D9B
:1003C00080830895EF92FF920F931F93CF93DF9353
:1003D000EC0181E0888F9B8D8C8D98131AC0E88981
:1003E000F989808185FF15C09FB7F894EE89FF8950
:1003F0006083E889F98980818370806480839FBFEE
:1004000081E090E0DF91CF911F910F91FF90EF90ED
:100410000895F62E0B8D10E00F5F1F4F0F731127FD
:10042000E02E8C8D8E110BC00FB607FCFACFE88939
:10043000F989808185FFF5CFCE01A2DFF2CFEB8D68
:10044000EC0FFD2FF11DE35AFF4FF0829FB7F89498
:100450000B8FEA89FB8980818062D0CF0F931F9335
:10046000CF93DF938C01D0E0C0E0F801EC0FFD1FCB
:100470006491662339F08BE994E0A4DF892B11F0B5
:100480002196F3CFCE01DF91CF911F910F91089567
:10049000CF93DF93EC01888D8823B1F0AA89BB89C3
:1004A000E889F9898C9185FD03C0808186FD0CC0A7
:1004B0000FB607FCF7CF8C9185FFF2CF808185FFC7
:1004C000EDCFCE015DDFEACFDF91CF9108958BE9CB
:1004D00094E041DF892BC9F08BE994E01ADF8C337B
:1004E00029F410927B0410927A04F1CF8A30C9F378
:1004F00080917A0490917B048436910594F701965B
:1005000090937B0480937A04E2CF089530DF8111C9
:10051000DEDF80E090E0892B49F080E090E0892BDD
:1005200029F00E94000081110E94000080E090E00C
:10053000892B49F080E090E0892B29F00E9400008F
:1005400081110E94000080E090E0892B49F080E05A
:1005500090E0892B29F00E94000081110C9400008A
:1005600008958150823108F05AC0E82FF0E08827C2
:10057000E354FD4F8F4F0C94CB0DDD02E102CF020F
:10058000D502D9020F03E402EA02EE02F402F802F5
:10059000FC02020306030F030A03100314038091F5
:1005A00080008F77809380000895809180008F7DF8
:1005B000F9CF80918000877FF5CF84B58F7784BD98
:1005C000089584B58F7DFBCF8091B0008F778093A5
:1005D000B00008958091B0008F7DF9CF8091900098
:1005E0008F77809390000895809190008F7DF9CF50
:1005F00080919000877FF5CF8091A0008F778093C6
:10060000A00008958091A0008F7DF9CF8091A00077
:10061000877FF5CF809120018F7780932001089507
:10062000809120018F7DF9CF80912001877FF5CFC8
:100630001F93CF93DF93282F30E0F901E254FE4F50
:100640008491F901E858FE4FD491F901EE5CFE4F18
:10065000C491CC23A1F0162F811183DFEC2FF0E0A1
:10066000EE0FFF1FE85EFE4FA591B4918FB7F8948F
:10067000EC91111108C0D095DE23DC938FBFDF9180
:10068000CF911F910895DE2BF8CFCF93DF9390E0A9
:10069000FC01E858FE4F24918E5C9E4FFC01849132
:1006A0008823C9F090E0880F991FFC01E250FF4FAA
:1006B000A591B491FC01E85EFE4FC591D491611102
:1006C0000DC09FB7F8948C91209582238C938881DC
:1006D000282328839FBFDF91CF910895623051F482
:1006E0009FB7F8943C91822F809583238C93E88167
:1006F0002E2BEFCF8FB7F894EC912E2B2C938FBF2E
:10070000EACF3FB7F8948091810490918204A09140
:100710008304B091840426B5A89B05C02F3F19F02F
:100720000196A11DB11D3FBFBA2FA92F982F882771
:10073000BC01CD01620F711D811D911D42E0660F4C
:10074000771F881F991F4A95D1F708958F929F921E
:10075000AF92BF92CF92DF92EF92FF924B015C017A
:10076000D0DF6B017C01CDDF6C197D098E099F09FB
:10077000683E734081059105B0F321E0821A91082B
:10078000A108B10888EEC80E83E0D81EE11CF11C58
:1007900081149104A104B10431F7FF90EF90DF9030
:1007A000CF90BF90AF909F908F9008952FB7F894FF
:1007B00060917D0470917E0480917F04909180040B
:1007C0002FBF0895FC01848187FD04C091E0692753
:1007D00063832EDF80E00895FC01808580FD04C0E6
:1007E00082FB882780F9089580E00895FC019085B8
:1007F000957081E0953009F080E00895862F642F90
:1008000044CFCF93DF93FC01218530E0F901E2541E
:10081000FE4F8491F901E858FE4FD491F901EE5C46
:10082000FE4FC491CC2371F081119BDEEC2FF0E0E0
:10083000EE0FFF1FEC51FF4FA591B491EC91ED230A
:1008400081E009F480E08170DF91CF910895DC01AF
:10085000ED91FD918081ED91FD919081ED91FD9162
:100860006C9163708E2309F064609F2309F06860C7
:10087000E4E4F4E0E60FF11D659565956D936D91E7
:100880007D918D919D91099423C01AC012C016C00C
:1008900010C01EC009C014C013C006C019C009C0D2
:1008A0000DC007C00DC014C0625070408040904021
:1008B0000BC0615070408040904006C06E5F01C028
:1008C0006F5F7F4F8F4F9F4F9E938E937E936E935C
:1008D0000895CF93DF93EC018B85823058F4F89420
:1008E000CE01B5DF6F81788589859A857894DF910F
:1008F000CF910895F894F6CF8F929F92AF92BF92C6
:100900000F931F93CF93DF93CDB7DEB7A1970FB6A9
:10091000F894DEBF0FBECDBF19A2423008F44AE002
:100920008E010F5D1F4F842E912CB12CA12CA5019F
:1009300094010E948D0DE62FB901CA01EA303CF501
:10094000E05DD801EE938D01232B242B252B79F725
:1009500090E080E0109761F0FD0101900020E9F740
:100960003197AF014A1B5B0BBD018BE994E095DC2D
:10097000A1960FB6F894DEBF0FBECDBFDF91CF9129
:100980001F910F91BF90AF909F908F900895E95C59
:10099000D8CF009761F0FC0101900020E9F7319772
:1009A000AF01481B590BBC018BE994E076CC90E079
:1009B00080E00895CF92DF92EF92FF920F931F9302
:1009C000CF93DF93EC01E62E84E090E00E94D30DFC
:1009D000FC0184E6808385E6818386E6828387E660
:1009E000838382E692E0998388838FEF8A838B8367
:1009F0008C838A878B878C8784E089878F016E013F
:100A000085E0C80ED11CF12CF80181918F0187FD82
:100A100032C0F60181936F0161E037DEF394F4E0B8
:100A2000FF12F2CF8FEF8C8388E692E09983888360
:100A30008B8587FD0FC0282F082E000C330BE21684
:100A4000130641F09A85913011F460E0F1DD60E029
:100A50008B851BDE82E08A87EB8662E08E2D15DEB9
:100A600081E08C87DF91CF911F910F91FF90EF90E4
:100A7000DF90CF900895F986D5CFCF93DF93EC0127
:100A800088819981009711F00E946F0E1982188257
:100A90001D821C821B821A82DF91CF910895FC0176
:100AA00080819181009711F00C946F0E08950E943F
:100AB000D40F0F931F93CF93DF93EC01888199811B
:100AC000009759F02A813B812617370730F081E0E3
:100AD000DF91CF911F910F9108958B016F5F7F4F31
:100AE0000E94F80E009759F0998388831B830A832C
:100AF0002C813D81232B59F7FC011082E8CF80E047
:100B0000E7CFEF92FF920F931F93CF93DF93EC0108
:100B10007B018A01BA01CDDF81110AC0CE01ADDFB0
:100B2000CE01DF91CF911F910F91FF90EF9008952B
:100B30001D830C83B701888199810E94E90FF0CF52
:100B40001F920F920FB60F9211240BB60F922F9394
:100B50003F934F935F936F937F938F939F93AF9345
:100B6000BF93EF93FF938BE994E00ADCFF91EF9141
:100B7000BF91AF919F918F917F916F915F914F91B5
:100B80003F912F910F900BBE0F900FBE0F901F90B3
:100B900018951F920F920FB60F9211240BB60F9259
:100BA0002F938F939F93EF93FF93E091AB04F0917A
:100BB000AC048081E091B104F091B20482FD1DC0CB
:100BC00090818091B4048F5F8F732091B504821758
:100BD00041F0E091B404F0E0E556FB4F958F80932F
:100BE000B404FF91EF919F918F912F910F900BBEC5
:100BF0000F900FBE0F901F9018958081F2CF1F921B
:100C00000F920FB60F9211242F933F938F939F93C0
:100C1000AF93BF9380917D0490917E04A0917F0457
:100C2000B091800430917C0423E0230F2D3758F5D8
:100C30000196A11DB11D20937C0480937D049093A7
:100C40007E04A0937F04B0938004809181049091EE
:100C50008204A0918304B09184040196A11DB11D6A
:100C60008093810490938204A0938304B0938404BE
:100C7000BF91AF919F918F913F912F910F900FBE98
:100C80000F901F90189526E8230F0296A11DB11D05
:100C9000D2CF1F920F920FB60F9211240BB60F9264
:100CA0002F933F934F935F936F937F938F939F9374
:100CB000AF93BF93EF93FF93809170049091710471
:100CC000C6DDFF91EF91BF91AF919F918F917F9181
:100CD0006F915F914F913F912F910F900BBE0F90AD
:100CE0000FBE0F901F9018951F920F920FB60F9284
:100CF00011240BB60F922F933F934F935F936F93F3
:100D00007F938F939F93AF93BF93EF93FF938091C4
:100D10006E0490916F049BDDFF91EF91BF91AF91B5
:100D20009F918F917F916F915F914F913F912F9103
:100D30000F900BBE0F900FBE0F901F9018951F9233
:100D40000F920FB60F9211240BB60F922F933F9371
:100D50004F935F936F937F938F939F93AF93BF93C3
:100D6000EF93FF93809178049091790470DDFF9167
:100D7000EF91BF91AF919F918F917F916F915F9113
:100D80004F913F912F910F900BBE0F900FBE0F9080
:100D90001F9018951F920F920FB60F9211240BB649
:100DA0000F922F933F934F935F936F937F938F9304
:100DB0009F93AF93BF93EF93FF93809176049091AD
:100DC000770445DDFF91EF91BF91AF919F918F9196
:100DD0007F916F915F914F913F912F910F900BBE3B
:100DE0000F900FBE0F901F9018951F920F920FB685
:100DF0000F9211240BB60F922F933F934F935F9353
:100E00006F937F938F939F93AF93BF93EF93FF93D2
:100E100080917404909175041ADDFF91EF91BF9158
:100E2000AF919F918F917F916F915F914F913F9182
:100E30002F910F900BBE0F900FBE0F901F90189523
:100E40001F920F920FB60F9211240BB60F922F9391
:100E50003F934F935F936F937F938F939F93AF9342
:100E6000BF93EF93FF938091720490917304EFDC32
:100E7000FF91EF91BF91AF919F918F917F916F9172
:100E80005F914F913F912F910F900BBE0F900FBE2E
:100E90000F901F90189590E0823090F40496833064
:100EA000910569F17CF481309105C9F00297F9F060
:100EB000809169008C7F816080936900E89A089531
:100EC0000297EDCF8430910511F1059789F7809154
:100ED0006A00837F846080936A00ED9A0895809110
:100EE0006900837F846080936900E99A0895809106
:100EF00069008F7C806180936900EA9A08958091EF
:100F000069008F73806480936900EB9A08958091E3
:100F10006A008C7F816080936A00EC9A089580E07B
:100F200008950F931F93CF93DF93EC01062F142F97
:100F300062E0802FAADB62E0812FA7DB802F90E0A8
:100F4000FC01EE5CFE4FE491F0E0EE0FFF1FEC5170
:100F5000FF4FA591B491B983A883FC01E858FE4FD7
:100F600024912C83812F90E0FC01EE5CFE4FE491F4
:100F7000F0E0EE0FFF1FEC51FF4F459154915B8362
:100F80004A83FC01E858FE4FE491ED831F821886E6
:100F900019861A868BE39FE10197F1F78C9128233C
:100FA00091E009F490E0DA018C91E82309F0926075
:100FB0009E83BE01802FB3DF082FBE01812FAFDFDC
:100FC000800F8B87DF91CF911F910F910895109221
:100FD0009E0410929D0488EE93E0A0E0B0E0809320
:100FE0009F049093A004A093A104B093A2048EE662
:100FF00092E090939C0480939B0485EC90E0909306
:10100000A8048093A70484EC90E09093AA048093B2
:10101000A90480EC90E09093AC048093AB0481EC45
:1010200090E09093AE048093AD0482EC90E09093B6
:10103000B0048093AF0486EC90E09093B204809368
:10104000B1041092B4041092B5041092B604109238
:10105000B704A8E3B5E090E080E041E2FC013E96F1
:1010600021E030E08630910510F430E020E0E20F1E
:10107000F31F40935700E491ED9301968930910559
:1010800069F762E686E696E095DC63E689E596E038
:1010900091DC4FE26EE289E196E043DF84E892E082
:1010A000909326068093250685E992E09093280682
:1010B0008093270641E360E389E296E032DF86EA27
:1010C00092E0909336068093350687EB92E09093FA
:1010D00038068093370643E362E389E396E021DF35
:1010E00088EC92E0909346068093450689ED92E065
:1010F000909348068093470645E364E389E496E0CD
:1011000010DF8AEE92E090935606809355068BEF9F
:1011100092E09093580680935706E7E4F5E020E8C4
:1011200032E08AE090E031832083128213821482BD
:10113000158297838683108611863E9646E0E931B4
:10114000F40789F710924205109241051092440568
:1011500010924305109246051092450550E040E07C
:1011600060E473E081E495E0CCCCCF93DF93CDB71E
:10117000DEB767970FB6F894DEBF0FBECDBF789489
:1011800084B5826084BD84B5816084BD85B582608C
:1011900085BD85B5816085BD80916E00816080933D
:1011A0006E001092810080918100826080938100A6
:1011B00080918100816080938100809180008160B6
:1011C000809380008091B10084608093B100809111
:1011D000B00081608093B000809191008260809324
:1011E00091008091910081608093910080919000A6
:1011F0008160809390008091A10082608093A10023
:101200008091A10081608093A1008091A000816005
:101210008093A000809121018260809321018091C0
:101220002101816080932101809120018160809360
:10123000200180917A00846080937A0080917A0006
:10124000826080937A0080917A00816080937A0036
:1012500080917A00806880937A001092C100E9E35F
:10126000CE2EE5E0DE2E8E010F5F1F4FD6018D9151
:101270006D011B861A861D861C861F861E8640E110
:10128000B80190E021D4F80101900020E9F73197EE
:10129000AF01401B510BB801CE010A9632DC1A8215
:1012A00019821C821B821E821D82609141057091F1
:1012B00042056115710531F0409145055091460593
:1012C000C8011FDCAA84BB84A114B10409F440C086
:1012D000EE84FF84E114F10499F08D819E81E80E83
:1012E000F91EB701C801E5DB882391F129813A8114
:1012F0008D819E81B501820F931F6BD6FE82ED8298
:1013000069817A816115710531F14D815E8181E4D8
:1013100095E0F7DBC801C3DBCE010A96C0DBB1E480
:10132000CB16B5E0DB0609F0A1CF00914105109185
:1013300042050115110599F0F8018081882379F0A3
:10134000082E000C990B34D6D8018D938D01F4CF63
:10135000C80193DBD5CF81E495E08FDBDBCF07E4D9
:1013600015E062E2C62E62E0D62E7AE0A72EB12CFE
:10137000F601F0807181D801ED91FC910280F3813A
:10138000E02D42E050E06F2DC8011995F801F1867B
:1013900010860190F081E02D0190F081E02DC801D0
:1013A0001995882339F0D80118968C911897836085
:1013B00018968C93FBD9F801628373838483958399
:1013C000B782A682F4E0CF0ED11C025F1F4F26E049
:1013D0000931120769F64BE9C42E44E0D42E0BE81C
:1013E00014E059E1E52E56E0F52EC70172DAD80176
:1013F0006D937D938D939D938D01B0E1EB0EF11C68
:10140000C016D10691F78CE093E08F51934031F4F0
:1014100061E08CE03AD961E08CE00AD968EE73E0D3
:1014200080E090E093D9E091AB04F091AC0482E0CD
:101430008083E091A704F091A8041082E091A904B0
:10144000F091AA0480E180831092B304E091AF048C
:10145000F091B00486E08083E091AD04F091AE0499
:10146000808180618083E091AD04F091AE04808141
:1014700088608083E091AD04F091AE048081806843
:101480008083E091AD04F091AE0480818F7D8083F4
:1014900082E390E0A0E0B0E080939F049093A004EA
:1014A000A093A104B093A20422242394312C7ED9CA
:1014B0002B013C018091180290911902A0911A020F
:1014C000B0911B02AC01BD014854544F6F4F7F4F88
:1014D000441655066606770630F4481659066A061D
:1014E0007B0608F03CC082E292E00E942E028CE073
:1014F00093E04FDA80E292E00E942E024AE062E03E
:1015000070E080E090E0F8D98EE192E00E942E0237
:1015100082E192E03EDA8CE192E00E942E0240915C
:1015200045055091460560914105709142058BE952
:1015300094E00E944D018AE192E00E942E024092C6
:1015400018025092190260921A0270921B02409285
:101550000E0250920F0260921002709211022BE85C
:10156000C22E24E0D22E09E116E0F12CE12CF1E0AC
:10157000F88B2CE033E02E52334009F0188AD80162
:101580001C968D919C91B3E081349B0709F428C18E
:101590008C54934009F424C1D8011E962D913C919E
:1015A00081E0B3E027353B0721F02256334009F0B4
:1015B00080E08888882009F415C1882309F412C1C5
:1015C000C80187D924E030E040E050E0C8D24901AA
:1015D0005A01F60180819181A281B3818815990514
:1015E000AA05BB050CF005C181E02091890430916A
:1015F0008A042130310509F080E0F8898F2341F019
:10160000809157069091580621E0E216F10421F0EE
:10161000D8011E968D919C91BCD988E192E00E94E0
:101620002E0240920E0250920F02609210027092AF
:101630001102F60181929192A192B1926F01FFEF96
:10164000EF1AFF0A005F1F4F24E0E216F10409F0D1
:101650008ECF42E252E05F8B4E8B07E415E0D12C37
:10166000C12C9CE0E92E93E0F92ED80118968C91BC
:1016700018978B7F18968C931897ED91FC91019099
:10168000F081E02DC80119958D8BF8018085869534
:1016900081708D88881609F4CEC088D8D80112963A
:1016A0006D937D938D939C93159718968C91B2E0D2
:1016B0008B27F8018087C8018FD8811105C0C80128
:1016C00095D8882309F47BC0BDE6EB16B3E0FB0692
:1016D00009F4EDC0E3E8EE16E3E0FE0609F4E7C026
:1016E000F9E9EF16F3E0FF0609F4E1C081E02EEA24
:1016F000E21623E0F20631F034ECE31633E0F306B1
:1017000009F080E0AE89BF898D909C9094012351AF
:10171000310991E02330310528F0BCE18B169104AA
:1017200009F090E0882309F4C4C0992309F4C1C0EA
:1017300040920A0250920B0260920C0270920D02CB
:101740001092880410928704AE89BF8912968D91F9
:101750009C911FD9C80140D8882309F4A1C182E116
:1017600092E00E942E02BBE28B169104D1F488888D
:101770008820B9F08091890490918A04009709F03B
:1017800086C130928A0420928904409200025092CD
:101790000102609202027092030261E080E00E9406
:1017A000180364E670E080E090E00E94A603409297
:1017B0000E0250920F0260921002709211022FEFEF
:1017C000C21AD20A025F1F4F4E895F894C5F5F4F7A
:1017D0005F8B4E8B5FE0C516D10409F046CFC2C0C7
:1017E00081E0E7CEC80175D822E030E040E050E06B
:1017F000EDCE88169906AA06BB060CF01ACF81E03A
:101800002091890430918A042130310509F080E06B
:10181000B8898B2341F08091550690915606E1E0FE
:10182000EE16F10421F0D8011C968D919C91B1D84F
:1018300086E192E0F4CE0E94D603D80112968D90F4
:101840009D90AD90BC9015979B01AC01281939096A
:101850004A095B0916968D919C91B0E0A0E028178B
:1018600039074A075B0708F426CFD80118968C91F0
:1018700081708D88881609F41ECF0E94D603D80186
:1018800012966D937D938D939C93159718968C91DA
:10189000B1E08B278460F80180870E94D603D801CD
:1018A0001A966D937D938D939C931D9704CF81E041
:1018B00029CFEDE6EE16E3E0FE0609F4E6C0F3E814
:1018C000EF16F3E0FF0609F4E0C029E9E21623E091
:1018D000F20609F4DAC081E03EEAE31633E0F306EB
:1018E00031F044ECE41643E0F40609F080E05AE1FC
:1018F0008516910409F028CF882309F425CF80911B
:101900000A0290910B02A0910C02B0910D02835833
:101910009F4FAF4FBF4F481659066A067B0610F11E
:101920003092880420928704D0928604C092850465
:1019300040920602509207026092080270920902D9
:10194000C8010E94EC03882321F010920502109236
:101950000402C8010E94F603882321F03092050298
:10196000209204028CE093E08E52934001F5809126
:10197000000290910102A0910202B09103028853EB
:101980009D4CAF4FBF4F84159505A605B70520F4B4
:1019900010928A04109289048091890490918A049B
:1019A00060E0892B09F061E080E00E9418038091DB
:1019B0000E0290910F02A0911002B0911102AC01A1
:1019C000BD014C595F4F6F4F7F4F44165506660659
:1019D000770628F4481659066A067B0660F48CE000
:1019E00092E00E942E0240920E0250920F026092EC
:1019F0001002709211028091060290910702A0914C
:101A00000802B091090283589F4FAF4FBF4F841512
:101A10009505A605B705B0F58091870490918804D7
:101A2000019781F5E0918504F0918604EE0FFF1F88
:101A3000EE0FFF1FEE5DFD4F828193810E94C9046E
:101A400080910402909105020097A9F588E092E048
:101A50000E942E0264E670E080E090E00E94A603FF
:101A600040920E0250920F02609210027092110288
:101A70001092880410928704E9E0F0E0F0930502E8
:101A8000E09304020E94860212CD81E030CF0197DC
:101A900009F087CE10928A041092890460E07ECE0D
:101AA000C8010E94F603882309F47BCE8EE092E001
:101AB0000E942E0276CE019769F684E092E0C8CFAC
:101AC00081E495E00C944F05BB27FB015527AA271D
:101AD000880F991FAA1FA41710F0A41B83955051BB
:101AE000B9F7A05DAA3308F0A95DA193009779F733
:101AF000B111B1931192CB0100C0DC01FC01672F41
:101B000071917723E1F7329704C07C916D937083D4
:101B10006291AE17BF07C8F30895A1E21A2EAA1B5F
:101B2000BB1BFD010DC0AA1FBB1FEE1FFF1FA2178D
:101B3000B307E407F50720F0A21BB30BE40BF50B8A
:101B4000661F771F881F991F1A9469F76095709513
:101B5000809590959B01AC01BD01CF010895052EA4
:101B600097FB16F400940FD057FD05D0D6DF07FC85
:101B700002D046F408C050954095309521953F4FCE
:101B80004F4F5F4F089590958095709561957F4F69
:101B90008F4F9F4F0895EE0FFF1F881F8BBF079039
:101BA000F691E02D19940F931F93CF93DF9382301A
:101BB000910510F482E090E0E0917506F0917606D0
:101BC00030E020E0B0E0A0E0309799F42115310535
:101BD00009F44AC0281B390B24303105D8F58A8115
:101BE0009B816115710589F1FB0193838283FE015D
:101BF00011C0408151810281138148175907E0F0DB
:101C00004817590799F4109761F012960C931297A0
:101C100013961C933296CF01DF91CF911F910F91B4
:101C200008950093750610937606F4CF21153105BB
:101C300051F04217530738F0A901DB019A01BD01A9
:101C4000DF01F801C1CFEF01F9CF909376068093C1
:101C50007506CDCFFE01E20FF31F819391932250C1
:101C6000310939832883D7CF2091730630917406C8
:101C7000232B41F420911E0230911F0230937406F1
:101C80002093730620911C0230911D02211531050D
:101C900041F42DB73EB74091200250912102241B00
:101CA000350BE0917306F0917406E217F307A0F488
:101CB0002E1B3F0B2817390778F0AC014E5F5F4FA2
:101CC0002417350748F04E0F5F1F5093740640935A
:101CD0007306819391939FCFF0E0E0E09CCFCF9388
:101CE000DF930097E9F0FC01329713821282A091F2
:101CF0007506B0917606ED0130E020E01097A1F472
:101D000020813181820F931F2091730630917406D8
:101D10002817390709F061C0F0937406E093730641
:101D2000DF91CF910895EA01CE17DF07E8F54A81E8
:101D30005B819E0141155105B1F7E901FB83EA83FF
:101D400049915991C40FD51FEC17FD0761F48081AB
:101D500091810296840F951FE9019983888382817E
:101D600093819B838A83F0E0E0E012968D919C91B1
:101D700013970097B9F52D913C911197CD010296DB
:101D8000820F931F2091730630917406281739072C
:101D900039F6309751F51092760610927506B09389
:101DA0007406A0937306BCCFD383C2834081518154
:101DB000840F951FC817D90761F44E5F5F4F888164
:101DC0009981480F591F518340838A819B81938356
:101DD00082832115310509F0B0CFF0937606E093A8
:101DE00075069ECFFD01DC01C0CF13821282D7CFD2
:101DF0004F925F926F927F928F929F92AF92BF921B
:101E0000CF92DF92EF92FF920F931F93CF93DF93C6
:101E10008C01009791F4CB01DF91CF911F910F912D
:101E2000FF90EF90DF90CF90BF90AF909F908F90FA
:101E30007F906F905F904F90B6CEFC01E60FF71F3A
:101E40009C0122503109E217F30708F4AAC0D90116
:101E5000CD91DC911197C617D70718F1C530D10580
:101E600070F0CE0104978617970748F0C61BD70B72
:101E70002297C193D1936D937C93CF0130DFC8013A
:101E8000DF91CF911F910F91FF90EF90DF90CF9056
:101E9000BF90AF909F908F907F906F905F904F908A
:101EA00008955B01AC1ABD0A4C018C0E9D1EA091D9
:101EB0007506B0917606512C412CF12CE12C10972F
:101EC00031F580917306909174068815990509F093
:101ED0005CC04616570608F058C080911C029091CD
:101EE0001D02009741F48DB79EB74091200250919A
:101EF0002102841B950BE817F90708F052C0F093F4
:101F00007406E0937306F90171836083B8CF8D91F5
:101F10009C91119712966C90129713967C90139740
:101F2000A815B90559F56C0142E0C40ED11CCA14BC
:101F3000DB0420F1AC014A195B09DA01129615970E
:101F400080F06282738251834083D9016D937C93C8
:101F5000E114F10471F0D7011396FC93EE931297FC
:101F60008ECF22968C0F9D1FF90191838083F30100
:101F7000EFCFF0937606E093750681CF48165906A9
:101F800008F42C017D01D3019ACFCB010CDE7C013A
:101F9000009739F0AE01B80113D0C801A0DE870167
:101FA0006ECF10E000E06BCF81E090E0F89418C0B5
:101FB0009111089581568A5108F4805285580895E8
:101FC000FB01DC0102C001900D9241505040D8F756
:101FD0000895FB01DC0101900D920020E1F70895C6
:101FE00011E0CBE1D1E000E005C0802FFE01D3DDA0
:101FF0002196011DCC31D10780E00807B1F7F89494
:02200000FFCF10
:10200200FFFFFFFF0900FFFFFFFFFFFFFFFFFFFFD3
:10201200FFFF332E312E3500FFFFFFFF0000770652
:1020220080001600DA031700E5031800ED0319001B
:10203200F8031A0001041B000D041C0019041D0002
:10204200240420002C042100340422003D04240036
:10205200450425004D041E0055041F0065040000C0
:102062000000570500000000E20300000000E2014A
:102072004D017A014802AB0189019D010000000077
:102082000104FE03454E435F464D535F4F55544591
:10209200525F444E00454E435F464D535F4F555489
:1020A20045525F555000454E435F464D535F494E82
:1020B2004E45525F444E00454E435F464D535F4985
:1020C2004E4E45525F555000454E435F434F4D5F64
:1020D200494E4E45525F444E00454E435F434F4D7D
:1020E2005F494E4E45525F555000454E435F434F48
:1020F2004D5F4F555445525F444E00454E435F433A
:102102004F4D5F4F555445525F5550005265616CBB
:1021120053696D476561722D474E53343330005217
:1021220065616C53696D476561722D473500526573
:10213200616C53696D476561722D47464335303096
:1021420000454E435F4844475F555000454E435F4C
:10215200414C545F555000454E435F4844475F44ED
:102162004E00454E435F414C545F444E0052656100
:102172006C53696D476561722D473130303050467E
:102182004431005265616C53696D476561722D4738
:10219200313030304D464431005265616C53696DC7
:1021A200476561722D4731303030584644005265E0
:1021B200616C53696D476561722D4731303030581B
:1021C200464431005265616C53696D476561722DF9
:1021D2004731303030584644320042544E5F4E410F
:1021E200565F46460042544E5F454E540042544E9E
:1021F2005F434F4D5F46460042544E5F4D454E553C
:102202000042544E5F5A4F4F4D5F444E0042544E6F
:102212005F5A4F4F4D5F55500042544E5F444952F2
:102222004543540042544E5F434C520042544E5F69
:102232004344490042544E5F50524F430042544E71
:102242005F4F42530042544E5F46504C0042544E40
:102252005F4D53470042544E5F4E41565F434F4DD0
:0E2262005F544F470042544E5F464D530000FC
:00000001FF
